:1000000008308A00DC2800000A108A100A118207D2
:1000100028340C3401340634D3346D38EC32202AC1
:10002000E832F236EF36653AE832F2060A00A831D5
:100030002910CB306B36E9352019B018B3060A0009
:10004000F73B77176D366131AE31FA060A00A831F9
:100050002910CB306B36E9352019B0183300F73B47
:1000600077176D366131AE317A00541DA0126610DB
:100070004B102000242A311730102533A0060A0027
:1000800083168613831286130830F8004728000071
:10009000F8175828F813B40C03188617031C861396
:1000A000781758287813F80B4B2856280000861725
:1000B0003F308400840B5A280000F81B4A28781B24
:1000C00052280800831603178C170C140000000038
:1000D00083120C087F390319A6280313A100031704
:1000E0000D080313A20003170F080313A300210830
:1000F000B4004020220803178D00031323080317C0
:100100008F0083168C170C140000000083120C0D56
:100110000E0D7F390319A6280313A10003170D083C
:100120000313A20003170F080313A3002108B40050
:100130004020220803178D000313230803178F00A4
:100140008D0A03198F0A031362280317031308008B
:1001500035308400831300080319BB280230F800EF
:10016000F701F70BB128F80BB0289730F700F70B21
:10017000B728800BAE2808003C18C0280812C128F8
:100180000816831608128312BC18C8288812C928BA
:1001900088168316881283123C19D0280813D12898
:1001A0000817831608138312BC19D8288813D92876
:1001B0008817831688130000831209148316091008
:1001C000E128E2288312091083160910831208001F
:1001D000BD018316081600308312081A0130BD04D1
:1001E0008316881600308312881A0130F700031036
:1001F000F70D7708BD048316081700308312081B1B
:100200000130F700F70DF70DFC30F7057708BD0456
:100210008316881700308312881B0130F700F70D12
:10022000F70DF70DF830F7057708BD043D08F80025
:10023000080083160910891009118312891083168A
:10024000891008168816081788178312091583164F
:10025000091100008312091483160910000083128B
:10026000E8207808BC0009108316091000008312EA
:100270000914831609103C298312E8207808BB0072
:1002800009108316091008128812081388138312A4
:100290003C0EF700F030F70577083B04F8007808CB
:1002A000BB00BB1F552983162129B908031D5A29F4
:1002B00089105B29891483168910000083120911A3
:1002C0008316091100008312091083160910831286
:1002D0003A0EBB000F30BB053B08BC00BC203A08FF
:1002E0000F39BB00BC00BC2008008316081288121E
:1002F00008138813091089100911831289108316B5
:1003000089108312091183160911831209108316AB
:1003100009100F308312B500A8200130A100210878
:10032000033C031C9B290330BC00BC200530B500F6
:10033000A820A10A8F290230BC00BC20A1012108FD
:10034000033C031CAC2921080420A200B9012208A7
:10035000BA001921A10A9F298A150A126129360BB0
:10036000B229B5294030B700B629B70101303502AE
:10037000B70737088038B800B9013808BA00192122
:1003800008003408073A0319CF290B3A0319D42976
:10039000063A0319DC29023A0319E229E729013058
:1003A000B500B600AF21ED29B9010130BA0019211D
:1003B0000230B500A820ED290130B5000230B600AA
:1003C000AF21ED29B9011030BA001921ED29013012
:1003D000B9003408BA001921ED2908008316031763
:1003E0008C170C140000000083120C087F390319CD
:1003F000322A0313A10003170D080313A2000317E9
:100400000F080313A3002108B400C1212208031719
:100410008D000313230803178F0083168C170C1409
:100420000000000083120C0D0E0D7F390319322AD3
:100430000313A10003170D080313A20003170F08ED
:100440000313A3002108B400C121220803178D0063
:100450000313230803178F008D0A03198F0A031350
:10046000EE290317031308000830AB02031C442ACB
:100470002B30840083130310800C00080319442AD6
:10048000422A0000800B412A0800A013200883168E
:100490008700831287130230AA00F830AB003422A1
:1004A000AA0B4D2AA017200883168700023083125A
:1004B000AA00F830AB003422AA0B592AA017200852
:1004C0008316870083120800AB012B08073C031C2E
:1004D0008B2AA01320088316870083128713702AA3
:1004E000712A0314AA0C0318772A8713782A87170E
:1004F000A0132008831687002730F700F70B7E2A09
:10050000812A8312A017200883168700872A882A49
:100510008312AB0A652A0800AA012A08073C031CBB
:10052000B42AA01320088316870083128713982A01
:10053000992AA0172008831687000530F700F70BCB
:100540009F2A8312A0172008831687008312871B17
:10055000AB2A0310AC2A0314AB0C4F30F700F70B97
:10056000AF2AB22AAA0A8D2A2B08F8000800A10196
:100570004522CC30AA0064224430AA006422A1089B
:10058000031DC62A8C227808A100BF2A4522CC3040
:10059000AA006422BE30AA0064228C227808A2003D
:1005A0008C227808A3002308A5002208A4002508AF
:1005B000AB002408AA008E30F7002B08F8002A08A8
:1005C000F900FA01AB1FE92AF809F909F90A031938
:1005D000F80AF808031DF62A7908F800F90108302E
:1005E000F702F808031DF62AF701FF2A0310F81B8B
:1005F000FD2AF90DF80DF703F62AAB1FF81377085B
:10060000AA007808AB007908AC007A08AD002D0884
:10061000B1002C08B0002B08AF002A08AE00B501CD
:10062000B401B3018330B2002E080319D92BBA00EC
:1006300032080319D92BBA02031C232B7F30BA07C7
:100640000318D92B292B8130BA02031CD92B03198B
:10065000D92B3A08F700F801F901FA01B9012F087E
:10066000B800B8173008B7003108B6001930BA0022
:100670003508B60203184C2B0130B70203184C2B77
:10068000B80203184C2BB90203184C2BB90AB80A4C
:10069000B70A3508B6077E2B3408B7020318672B54
:1006A0000130B8020318672BB9020318672BB90A87
:1006B000B80A3408B7073508B607031C7E2BB70AFB
:1006C000031D7E2BB80A031D7E2BB90A7E2B33082F
:1006D0008038B80203187D2B0130B90203187D2B36
:1006E000B90A33088038B8073408B707031C5B2BF6
:1006F000B80A031D5B2BB90A5B2B7A14BA0B812B4A
:100700008C2B0310B60DB70DB80DB90D0310FA0DF3
:10071000F90DF80DBB0D382B3B1C942B0310F80C76
:10072000F90CFA0CBB0C972BF7030319D92BBB1B45
:10073000C02B0310B60DB70DB80DB90D3508B602B4
:100740000318AC2B0130B7020318AC2BB802031806
:10075000AC2BB902031CCF2B3408B7020318B72BFC
:100760000130B8020318B72BB902031CCF2B330892
:100770008038B8020318C02B0130B902031CCF2BFC
:10078000FA0A031DCF2BF90A031DCF2BF80A031D0C
:10079000CF2BF70A0319D92BF80CF90CFA0C2F08F8
:1007A000BA003308BA06BA1FD72BF817DD2BF81397
:1007B000DD2BF701F801F901FA017A08A90079089F
:1007C000A8007808A7007708A6002608F7002708E1
:1007D000F8002808F9002908FA000800803083187A
:1007E000AC06B101B2012808B0002C08B0062708F9
:1007F0000319DE2CAF00F7002B080319E72CAF021A
:100800000319832C031C412C2C08B500B5172D08A7
:10081000B4002E08B300B2010310B50CB40CB30C35
:10082000B20CAF0B0B2CB01F182C3114FB2C311059
:100830002F1031162A3084008313102D3112B01B73
:100840002B2C2F1C362CB50CB40CB30CB20CF70AA5
:100850000319F62C362CB51B392C0310B20DB30D31
:10086000B40DB50DF7030319F62C2B2C3117A32C5F
:1008700031132808B000B01F3F2CB517EF2CB5136B
:10088000EF2C2B08AF00F7002708AF022808B500AF
:10089000B5172908B4002A08B300B2010310B50C3B
:1008A000B40CB30CB20CAF0B4D2CB01F5A2CB114BE
:1008B000FB2CB1102F10B1162E3084008313102D95
:1008C000B112B01B6D2C2F1C782CB50CB40CB30CD2
:1008D000B20CF70A0319F62C782CB51B7B2C0310ED
:1008E000B20DB30DB40DB50DF7030319F62C6D2C35
:1008F000B117A32CB1132C08B000B01F812CB51771
:10090000EF2CB513EF2C2C08B500B5172D08B4004B
:100910002E08B300B01F902CB5133115FB2C3111EC
:10092000B2012F102A3084008313102DB01BB92C74
:100930002808B0002F1CA32CB50CB40CB30CB20CBF
:10094000F70A0319F62CB21FB42CB30A031DB42CFA
:10095000B40A031DB42CB50A031DB42CB50CB40C99
:10096000B30CF70A0319F62C311B382CB11B7A2C67
:10097000D82C8030B506B51FC12CFB2C2C08B0003C
:10098000CE2C2808B000B508031DCE2CB408031DDA
:10099000CE2CB308031DCE2CF701EF2CB51BD82CA1
:1009A0000310B20DB30DB40DB50DF70BCE2CF62C14
:1009B000B01FDC2CB517EF2CB513EF2C2B08F7006C
:1009C0002C08B5002D08B4002E08B300EF2C270822
:1009D000F7002808B5002908B4002A08B300350834
:1009E000F8003408F9003308FA002E2DF701F80159
:1009F000F901FA012E2DB201B309B409B509B20902
:100A0000B20A031D092DB30A031D092DB40A0319E7
:100A1000B50A3118172CB118592C31198F2CBE2C4E
:100A20000008B307031C1A2DB40A031D1A2DB50ABA
:100A300003192F1484030008B407031C222DB50AE0
:100A400003192F1484030008801F803AB507031888
:100A50002F14311A1E2CB11A602C962C0800340861
:100A600003199F2DBC00380803199F2DBC070318DC
:100A7000402D7F30BC02031C9F2D03199F2D442D58
:100A80008130BC0703189F2D3C08F700F801F901DD
:100A9000FA013508C000C0173608BF003708BE008D
:100AA0001830BC00BD013E1C6D2D3B08FA07031C2D
:100AB0005F2DF90A031D5F2DF80A0319BD173A08C7
:100AC000F907031C662DF80A0319BD173908B6008B
:100AD000B6173608F8070318BD17BD0DF80CF90C4A
:100AE000FA0CC00CBF0CBE0C0310BC0B522D013015
:100AF000F70703189F2DF81B842DC00DFA0DF90D73
:100B0000F80DF70303199F2DC01F952DFA0A031D39
:100B1000952DF90A031D952DF80A031D952DF80C46
:100B2000F90CFA0CF70A03199F2D3508BD00390896
:100B3000BD06BD1F9D2DF817A32DF813A32DF7019A
:100B4000F801F901FA0108003408B63CB400FA01D2
:100B50003508B800B5170310B50CB60CB70CFA0C75
:100B6000F90CF80CF70CB40BAB2DB81FC22DF7091C
:100B7000F809F909FA09F70A0319F80A0319F90A31
:100B80000319FA0A0800F701F801F901FA01BC019A
:100B9000BD01BE01BF013B083A0439043804031902
:100BA000012E2030C0000310B40DB50DB60DB70DE9
:100BB000BC0DBD0DBE0DBF0D3B083F02031DEA2D50
:100BC0003A083E02031DEA2D39083D02031DEA2DB5
:100BD00038083C02031CFB2D3808BC023908031CF2
:100BE000390FBD023A08031C3A0FBE023B08031C32
:100BF0003B0FBF020314F70DF80DF90DFA0DC00BF2
:100C0000D32D3C308400831308000408AC002B086B
:100C1000AE000319242E2A08B7002908B6002808B8
:100C2000B5002708B400BB01BA012030B9008230FA
:100C3000B8002F257A08AA007908A9007808A8002A
:100C40007708A700AE0B0B2E2A08B7002908B600BC
:100C50002808B5002708B400A4257A08AA00790856
:100C6000A9007808A8007708A700AA1F442EAC03A3
:100C7000AC16A709A809A909AA09A70A0319A80A6D
:100C80000319A90A0319AA0A3B30B3009A30B2002B
:100C9000CA30B100B0010A30AE002B080319AC0A0B
:100CA0002A08B7002908B6002808B5002708B400AC
:100CB0003308BB003208BA003108B9003008B80068
:100CC000C3250008A700840A0008A800840A0008B9
:100CD000A900840A0008AA00FD308407F708031D54
:100CE000842E2B0A2E020319842E2C080319862E1B
:100CF0000F392E0203197E2E0318B62EAC1BB62E0A
:100D00002C1B862E2030B22E2030AC05AC1E942E2B
:100D1000AC122B08031DAC037708AC002D30B400D7
:100D2000C1212C08F700AC012B082E02031DA22EB6
:100D30007708AC002E30B400C1212C08F700203019
:100D4000AC0500303030AC1EB22EAC122B08031DA7
:100D5000AC037708AC002D30B400C1212C08F7009B
:100D6000AC013030F7077708B400C1213308B70071
:100D70003208B6003108B5003008B400BB01BA0132
:100D8000B9010A30B800C3257A08B3007908B20067
:100D90007808B1007708B000AE0B502E8A150A1201
:100DA000DA29831603178C170C14000000000318AF
:100DB000002F83120C087F390313A80003170D08B6
:100DC0000313A90003170F080313AA002808B4008F
:100DD000C121290803178D0003132A0803178F0068
:100DE00083168C170C140000000083120313A70B4A
:100DF000FA2EFD2E83160317002F1F2F83160317BD
:100E000083120C0D0E0D7F390313A80003170D0874
:100E10000313A90003170F080313AA002808B4003E
:100E2000C121290803178D0003132A0803178F0017
:100E30008D0A03198F0A03100313A70BD12E8A15ED
:100E40000A12E629831603178C170C140000000001
:100E50000318512F83120C087F390313A8000317BE
:100E60000D080313A90003170F080313AA0028088D
:100E7000B4004020290803178D0003132A08031724
:100E80008F0083168C170C140000000083120313CC
:100E9000A70B4B2F4E2F83160317512F702F83163E
:100EA000031783120C0D0E0D7F390313A8000317CF
:100EB0000D080313A90003170F080313AA0028083D
:100EC000B4004020290803178D0003132A080317D4
:100ED0008F008D0A03198F0A03100313A70B222F0B
:060EE0008A150A12242A03
:101000000408AC002B08AE00031921282A08B700F9
:101010002908B6002808B5002708B400BB01BA01AA
:101020002030B9008230B8008A112F258A157A083D
:10103000AA007908A9007808A8007708A700AE0BD5
:1010400006282A08B7002908B6002808B50027088E
:10105000B4008A11A4258A157A08AA007908A90083
:101060007808A8007708A700AA1F4328AC03AC168D
:10107000A709A809A909AA09A70A0319A80A03190F
:10108000A90A0319AA0A3B30B3009A30B200CA3049
:10109000B100B0010A30AE002B080319AC0A2A08CF
:1010A000B7002908B6002808B5002708B40033089F
:1010B000BB003208BA003108B9003008B8008A1104
:1010C000C3258A150008A700840A0008A800840A1E
:1010D0000008A900840A0008AA00FD308407F70868
:1010E000031D85282B0A2E02031985282C080319B5
:1010F00087280F392E0203197F280318BF28AC1B3D
:10110000BF282C1B87282030B9282030AC05AC1E06
:101110009728AC122B08031DAC037708AC002D30C8
:10112000B4008A1140208A152C08F700AC012B0866
:101130002E02031DA7287708AC002E30B4008A11B8
:1011400040208A152C08F7002030AC0500303030E4
:10115000AC1EB928AC122B08031DAC037708AC00F9
:101160002D30B4008A1140208A152C08F700AC01FC
:101170003030F7077708B4008A1140208A15330809
:10118000B7003208B6003108B5003008B400BB0122
:10119000BA01B9010A30B8008A11C3258A157A0844
:1011A000B3007908B2007808B1007708B000AE0B40
:1011B0004F288A150A12322A840183131F308305AF
:1011C000713083168F000F088613831286178316DB
:1011D00003170908C039890003131F129F1200303A
:1011E000031788008312870188018901FF300313E8
:1011F000A000831603170908C039890003131F12C2
:101200009F12003003178800831203131F139F13CC
:1012100083169F1783121F149412A012200883169E
:101220008700831220162008831687008312A011DE
:101230002008831687000130831294000030831643
:1012400094000108C73908388100831290010030EA
:10125000F8009200003083169200831220152008B7
:10126000831687008312970183169B019C0101302E
:101270009D0083120317870188018901713083164D
:1012800003138F000F080C30831203178D000030FA
:101290008F008A11031362208A15173003178D00FF
:1012A00000308F008A11031362208A152030031743
:1012B0008D0000308F008A11031362208A158A1175
:1012C00075298A15273003178D0000308F008A1189
:1012D0000313EE218A150330B5000230B6008A11DF
:1012E000AF218A152F3003178D0000308F008A112F
:1012F0000313EE218A150830A100FA30B5008A11D7
:10130000A8208A15A10B7D290130B5000230B60056
:101310008A11AF218A158A11B7228A157708A10090
:101320007808A2007908A3007A08A400A60104089E
:10133000A5002610831B261483107A08AA007908BA
:10134000A9007808A8007708A7003330AE009330D2
:10135000AD000830AC008730AB008A11EE238A154F
:10136000250884008313261883177708A1007808BE
:10137000A2007908A3007A08A4005430B4008A11AE
:10138000C1218A153A30B4008A11C1218A15203052
:10139000B4008A11C1218A15893084002408AA006A
:1013A0002308A9002208A8002108A7000230AB00EA
:1013B0008A11052E8A15373003178D0000308F00F3
:1013C000031404300313A7008A11D12E8A158A1141
:1013D000B7228A157708A1007808A2007908A3002F
:1013E0007A08A400A6010408A5002610831B261471
:1013F00083107A08AA007908A9007808A80077085D
:10140000A7003330AE009330AD000830AC00873019
:10141000AB008A11EE238A15250884008313261851
:1014200083177708A1007808A2007908A3007A083A
:10143000A4003A3003178D0000308F0003100630EF
:101440000313A7008A11222F8A15893084002408EB
:10145000AA002308A9002208A8002108A70002303A
:10146000AB0000282030B4008A1140208A150D30CE
:10147000B4008A1140208A150A30B4008A11402035
:101480008A156430B5008A11A8208A158429630062
:04400E00F52CFF3F4F
:00000001FF
